:1000000012C02BC02AC08DC028C027C026C025C062
:1000100024C023C022C021C020C01FC01EC01DC0DC
:100020001CC01BC01AC011241FBECFE5D4E0DEBF28
:10003000CDBF10E0A0E6B0E0E6E4F1E002C005903C
:100040000D92A036B107D9F710E0A0E6B0E001C0EC
:100050001D92A036B107E1F729C0D2CF40E050E0B1
:100060004817590768F420E030E0275E3F4F60E70B
:100070002E343607D0F34F5F5F4F4817590798F378
:10008000089587B38F6387BB88B3807F806388BB05
:1000900084B3837C836084BB85B3807C85BB81B360
:1000A00086EF81BB82B382E282BB0895CFE5D4E0C4
:1000B000DEBFCDBFE6DF919A85B589E185BD83B509
:1000C0008E6683BD89B78278806889BF8FB7806864
:1000D0008FBF88B3866088BB88B3897F88BB89B7A8
:1000E000806889BF84E690E0B9DF809908C082B358
:1000F0008F7D806182BB88B38F7D806107C082B3B2
:100100008F7E806282BB88B38F7E806288BB89B716
:100110008F7789BF88B3866088BB84E690E09EDFD6
:10012000DBCF1F920F920FB60F9211248F939F93E4
:1001300082B390E8892782BB9F918F910F900FBE69
:060140000F901F901895BE
:00000001FF
